:100000000C9434000C9451000C9451000C94510049
:100010000C9451000C9451000C9451000C946E0CF3
:100020000C9451000C94E4010C9451000C94DC08E5
:100030000C9451000C9412090C9451000C94510032
:100040000C9451000C9451000C9451000C945100EC
:100050000C9451000C9451000C9451000C945100DC
:100060000C9451000C94510011241FBECFEFD4E02A
:10007000DEBFCDBF11E0A0E0B1E0EAE5FCE102C0E7
:1000800005900D92AC30B107D9F712E0ACE0B1E0C9
:1000900001C01D92A937B107E1F70E9468070C94CF
:1000A0002C0E0C9400008F929F92AF92BF92CF9231
:1000B000DF92EF92FF920F931F93CF93DF93B82EAF
:1000C0006B01F42E07DAA82E6B2D8DE090E0AAD9F3
:1000D0008C016B2D87E690E0A5D9EC01812E992447
:1000E000882D8F3709F020C10068003AD9F493E0D9
:1000F000D694C7949A95E1F7EB2DF0E0EE0FFF1F31
:10010000E45FFE4F80819181C816D90629F48B2DBA
:10011000C0D9882309F4FFC04D2F55272C2D6A2DF7
:1001200080EA4BC0003DD1F413E0D694C7941A95F1
:10013000E1F7EB2DF0E0EE0FFF1FE45FFE4F808153
:100140009181C816D90629F48B2DA3D9882309F4E7
:10015000E2C04C2D6A2D80ED24D9DDC0003EE9F4CB
:10016000EB2DF0E0EE0FFF1FE45FFE4F80819181E9
:10017000C816D90629F48B2D8CD9882309F4CBC055
:10018000960173E0369527957A95E1F74C2D4770E7
:100190004295407F6A2D80EE10C00039E9F4FF20BF
:1001A00071F06B2D87E690E03DD9092F11278B2D3B
:1001B00091D92C2D402F682F80E9E2D8ACC06B2D4F
:1001C00087E690E02FD9092F11278B2D83D92C2D6D
:1001D000402F682F80E8F1CF0A3F21F4FF2049F03B
:1001E0008AEF05C00B3F39F4FF2019F08BEF6FD871
:1001F00092C08CEFFCCF0139A1F5E60143E0D69522
:10020000C7954A95E1F70B2D10E0F801EE0FFF1F9F
:10021000E45FFE4F8081918123E0969587952A9532
:10022000E1F7C817D90729F48B2D33D9882309F4AE
:1002300072C08BE8E82E81E0F82EE00EF11EF70187
:1002400010818B2D47D920E0412F682F80E898D866
:100250008B2D40D92FE74C2F682F80E991D8F701DB
:1002600030C0023981F5E601B3E0D695C795BA955D
:10027000E1F70B2D10E0F801EE0FFF1FE45FFE4FDA
:1002800080819181F3E096958795FA95E1F7C817FB
:10029000D90721F48B2DFDD88823E9F18B2D1AD9AC
:1002A0002FE74C2F682F80E96BD805571E4FF801B8
:1002B000F0808B2D0FD920E04F2D682F80E860D87B
:1002C000F801C08328C0033909F071C08601E3E05A
:1002D00016950795EA95E1F7CB2DD0E0FE01EE0FDC
:1002E000FF1FE45FFE4F8081918163E096958795C3
:1002F0006A95E1F70817190721F48B2DCAD88823CE
:1003000051F08B2DE7D82FE7402F682F80E938D8A0
:10031000C557DE4F0883EB2DF0E0EE0FFF1FE45FC3
:10032000FE4FD182C08243C0760143E0F694E79449
:100330004A95E1F7CB2DD0E0FE01EE0FFF1FE45F01
:10034000FE4F8081918123E0969587952A95E1F76C
:10035000E816F90621F48B2D9CD8882329F02E2D40
:10036000482D6A2D80EB0CD80F37D9F0FE01EE0F27
:10037000FF1FE45FFE4F80819181960127703070EE
:10038000877090702817390721F48B2D82D8882325
:1003900041F02C2D27702295207F402F6A2D80EB75
:1003A000EFD7CC0FDD1FC45FDE4FD982C882DF914B
:1003B000CF911F910F91FF90EF90DF90CF90BF9062
:1003C000AF909F908F9008951F920F920FB60F924B
:1003D00011242F923F924F925F927F928F929F9221
:1003E000AF92BF92CF92DF92EF92FF920F931F9343
:1003F0002F933F934F935F936F937F938F939F932D
:10040000AF93BF93EF93FF93CF93DF93CDB7DEB757
:100410002297DEBFCDBF85E082BF3699C2C204B14C
:1004200015B177B027E0722234E0371510F417B811
:1004300003C0739477B87A9467B1677082E090E0F4
:100440003DD8823008F4369A672D82E090E036D8A5
:10045000823008F0A6C28130A9F483E0003F18077B
:1004600088F0E72DF0E0EE0FFF1FEE0FFF1FED5AB3
:10047000FE4F8FEF9FEFAFEFBFEF80839183A2839B
:10048000B3831FC0E72DF0E0EE0FFF1FEE0FFF1F3D
:10049000ED5AFE4F20813181428153812F3F9FEFE2
:1004A00039079FEF49079FEF590759F0C801A0E0AE
:1004B000B0E0280F391F4A1F5B1F2083318342831E
:1004C0005383872C9924F401E85CFE4F90819F5F51
:1004D0009083F401E158FE4F80818F3710F48F5FD5
:1004E0008083929596959770840104551E4FF8016C
:1004F0008081891708F055C2C2D721E030E0082C6E
:1005000002C0220F331F0A94E2F73A832983822321
:100510009323892B09F429C27401EE0CFF1CEE0C05
:10052000FF1C83E591E0E80EF91EF70160817181FF
:10053000828193816F3FFFEF7F07FFEF8F07FFEF10
:100540009F0709F4E3C125E0969587957795679510
:100550002A95D1F7F801208130E02F5F3F4F4427E3
:1005600037FD4095542F38DBF701208331834283D8
:100570005383672D8DE090E055D71C0160E0872DF7
:1005800067D76C0161E0872D63D72C0162E0872D6E
:100590005FD75C018C159D0570F4C601A0E0B0E04A
:1005A0008093230190932401A0932501B093260109
:1005B000C50156016C01F7012081318142815381CF
:1005C0002093230130932401409325015093260169
:1005D000720100E010E02E153F054007510730F48E
:1005E000F401E85BFE4F808181600AC0E216F306E9
:1005F0000407150730F4F401E85BFE4F8081826048
:100600008083F401EE0FFF1FEA56FE4F0190F08148
:10061000E02DE415F50530F4E216F306040715079E
:1006200048F00DC04E165F0650F42E153F054007EA
:10063000510728F4F401E158FE4F81E08083832DB7
:1006400099278F37910509F0FFC00FE7E02EF12CB5
:10065000E220F32080E890E0E82AF92A90E9E91600
:10066000F10449F0EAEFEE16F10429F0FBEFEF1682
:10067000F10409F0E9C0C601A0E0B0E0281739078D
:100680004A075B0708F06CC0F401E85BFE4F80810D
:1006900081FF66C08091430190E0082C02C09595CF
:1006A00087950A94E2F780FF5BC060E0872DD0D683
:1006B0008C0162E0872DCCD60817190700F520E9D8
:1006C000E216F10469F030E9E316F104D8F186E0AE
:1006D0009FEFE80EF91E92E0E916F10498F50DC0BF
:1006E000672D87E690E09ED6092F1127872DF2D639
:1006F00024E6402F682F80E81AC08CEF22C0EAEF72
:10070000EE16F104D9F0FBEFEF16F104C9F020E981
:10071000E216F104B9F4672D87E690E083D6092F3D
:100720001127872DD7D624E6402F682F80E928D6B9
:10073000F401E158FE4F80E8808304C08AEF01C0D5
:100740008BEFC5D5F401E85BFE4F80818D7F808300
:100750009981909580914301892380934301D6C06C
:10076000C501A0E0B0E082179307A407B50708F021
:10077000CDC0F401E85BFE4F808180FFC7C080914F
:10078000430190E0082C02C0959587950A94E2F702
:1007900080FDBCC060E0872D5BD68C0162E0872DB8
:1007A00057D608171907E8F43AEFE316F104A9F051
:1007B0008BEFE816F10499F090E9E916F104B9F528
:1007C000672D87E690E02ED6092F1127872D82D638
:1007D00024E6402F682F80E921C08AEF27C08BEFE5
:1007E00025C0E0E9EE16F10469F0F0E9EF16F10436
:1007F000F0F026E03FEFE20EF31E32E0E316F104E4
:10080000B0F413C0672D87E690E00CD6092F1127AE
:10081000872D60D624E6402F682F80E8B1D5F401FB
:10082000E158FE4F80E8808302C08CEF50D5809164
:1008300043019981892B80934301F401E85BFE4FCA
:1008400080818E7F808362C0C601A0E0B0E028175F
:1008500039074A075B0748F41092230110922401DC
:1008600010922501109226010CC0281B390B4A0B4F
:100870005B0B209323013093240140932501509377
:1008800026016091230170912401809125019091AE
:100890002601EAE0660F771F881F991FEA95D1F7B6
:1008A000AC18BD08950140E050E096D92093230193
:1008B0003093240140932501509326012050344069
:1008C0004040504060F08FEF93E0A0E0B0E08093B4
:1008D000230190932401A0932501B0932601E09079
:1008E0002301F090240160E0872DB2D58C0162E0F5
:1008F000872DAED58017910728F48FEF93E08E19DE
:100900009F097C0140E0B701872DCDDB10910001EC
:10091000171559F589E68093B70181E38093B801F3
:100920004BD58F5F8093B9011093BA01F401EE0F9C
:10093000FF1FEE0FFF1FED5AFE4F80819181A281B4
:10094000B3819C01AD0163E0569547953795279596
:100950006A95D1F72093BB0187708295807F809341
:10096000BC0186E080932901EDD4F401EE0FFF1F56
:10097000EA56FE4FD401AA0FBB1FAA0FBB1FAD5AE8
:10098000BE4F8D919C911197918380831D921D92F2
:100990001D921C92139728E331E0820E931EF401FE
:1009A00010822296F894DEBFCDBFDF91CF91FF91E8
:1009B000EF91BF91AF919F918F917F916F915F91D7
:1009C0004F913F912F911F910F91FF90EF90DF90EA
:1009D000CF90BF90AF909F908F907F905F904F90FF
:1009E0003F902F900F900FBE0F901F9018951F9360
:1009F000CF93DF9380912901815080932901823028
:100A000020F08091B7018D3719F0109229015CC256
:100A100089E68093B7011091B801103409F458C1E8
:100A2000113428F5153109F496C0163180F41031CF
:100A300009F472C0113120F4113009F045C23CC0F4
:100A4000123109F446C0133109F03EC28EC0123291
:100A500009F493C0133220F4103209F035C2C4C037
:100A6000103309F4DDC0123309F02EC2E6C012368D
:100A700009F4A6C1133680F4103509F48BC1113581
:100A800020F4123409F020C2E6C0123509F460C126
:100A9000103609F019C2B0C1153609F4C4C11636B2
:100AA00020F4133609F010C2D8C1163609F4F5C186
:100AB000183609F009C2E8C182E08093B8017CD4FD
:100AC0008F5F8093B90183E08093BA011093BB01DB
:100AD0003EC072D490E001962091B90130E08217B7
:100AE000930709F0F1C14091BB0150E0542F442716
:100AF0008091BC0190E0482B592B6091BA01615064
:100B00008DE090E0F8D4E091BA01F0E0EE0FFF1F25
:100B1000E65FFE4F118210824FD490E00196209143
:100B2000B90130E08217930709F0CEC181E18093CB
:100B3000B80142D48F5F8093B9016091BA016150CE
:100B40008DE090E06FD4292F33272093BB01809351
:100B5000BC0186E0B6C14091BB016091BA0182E060
:100B600090E06ED48091BA014DD684E18093B801B3
:100B70006091BA0182E090E054C11ED490E00196E9
:100B80002091B90130E08217930709F09DC180914F
:100B9000BB0190E09695982F88279795879520918F
:100BA000BA0130E0822B932B6FD4C0E0D0E0FE017D
:100BB000EE0FFF1FE45FFE4F1182108260D421E030
:100BC00030E00C2E02C0220F331F0A94E2F72823D4
:100BD0003923232B19F08C2F15D602C0CE019DD5B9
:100BE0002196CB30D10519F7E7D390E001962091FB
:100BF000B90130E08217930709F066C181E2809362
:100C0000B801DAD38F5F8093B90139D4282F2F77B9
:100C10002093BA01880F892F881F990B919530C1B5
:100C2000CBD390E001962091B90130E08217930771
:100C300009F04AC18091BA010BC0BED390E0019681
:100C40002091B90130E08217930709F03DC18FEF81
:100C50008093000139C1B0D390E001962091B90191
:100C600030E08217930709F02FC12091BF0130E0D7
:100C70003695322F2227379527958091C00190E035
:100C8000282B392B4091BD0150E05695542F442715
:100C9000579547958091BE0190E0482B592B609164
:100CA000BB0170E07695762F6627779567958091E2
:100CB000BC0190E0682B792B8091BA0127D4E09198
:100CC000BA01F0E0EE0FFF1FE45FFE4F11821082C9
:100CD00073D390E001962091B90130E08217930719
:100CE00009F0F2C081E48093B80166D38F5F8093EE
:100CF000B90160E08091BA01ABD39C01220F232F90
:100D0000221F330B31952093BB018F778093BC0159
:100D100061E08091BA019CD39C01220F232F221FF6
:100D2000330B31952093BD018F778093BE0162E034
:100D30008091BA018DD39C01220F232F221F330BE8
:100D400031952093BF018F778093C0018AE0B9C0AD
:100D500033D390E001962091B90130E082179307D8
:100D600009F0B2C04091BB0150E0542F442780915C
:100D7000BC0190E0482B592B6091BA0187E690E0C6
:100D8000BAD3E091BA01F0E0EE0FFF1FE45FFE4F2F
:100D90001182108211D390E001962091B90130E0C8
:100DA0008217930709F090C081E58093B80104D3BE
:100DB0008F5F8093B9016091BA0187E690E0C2CE5F
:100DC000FBD290E001962091B90130E082179307A1
:100DD00009F07AC04091BB016091BA018DE790E0C3
:100DE0002FD31091BA01612F8DE790E067D3E12FE7
:100DF000F0E0E455FE4F8083DFD290E00196209131
:100E0000B90130E08217930709F05EC081E6809354
:100E1000B801D2D28F5F8093B9016091BA018DE79A
:100E200090E04CD32DC0C8D290E001962091B9013A
:100E300030E08217930709F047C04091BB016091F1
:100E4000BA0188E890E0FCD2E091BA01F0E0EE0F40
:100E5000FF1FE45FFE4F11821082AED290E0019638
:100E60002091B90130E08217930771F584E68093F1
:100E7000B801A2D28F5F8093B9018091BA012AD3C1
:100E80008093BB0185E01DC097D290E00196209130
:100E9000B90130E082179307B9F48ED290E0019641
:100EA0002091B90130E08217930771F487E68093AF
:100EB000B80182D28F5F8093B901FAD28093BA01D0
:100EC00084E0809329013ED2DF91CF911F91089554
:100ED0008F929F92AF92BF92CF92DF92EF92FF924A
:100EE0000F931F93CF93DF93D2D48DE390E05BD128
:100EF00063D280938A0122D323E5E22E21E0F22EF1
:100F0000C0E0D0E00DE710E0FE01E85CFE4F10828B
:100F1000F70111921192119211927F016C2FC80169
:100F2000CDD2FE01E455FE4F80832196C630D10517
:100F300059F71AD3C0E0D0E0A2D221E030E00C2E65
:100F400002C0220F331F0A94E2F728233923232BF0
:100F500019F08C2F57D402C0CE01DFD32196CB30AD
:100F6000D10551F77894109229011092220191E055
:100F7000A92E91E0B92E82E0882E80E0982E0DE017
:100F8000C02E00E0D02E7CD1892BE9F385D1AC01B5
:100F9000282F87FF30C0883FD9F0893F28F4803F51
:100FA00039F0873FE9F40DC08A5F8330C8F410C080
:100FB000109222011092290181E080932B0188EF89
:100FC00005C010922B011092220183EF80D139C00D
:100FD000109229012093440181E0809322012FC0C7
:100FE000109229012093440181E08093220183E043
:100FF00080932B0126C080912B01813059F4809180
:101000002901E82FF0E0E954FE4F40838F5F809381
:10101000290117C08330A9F480912201E82FF0E064
:10102000EC5BFE4F4083982F9F5F9093220180914D
:101030004401803D11F4923011F0933011F410927C
:101040002B0180912B01882309F09DCF80912901EC
:10105000882311F0CCDC97CF80912201882309F4FA
:1010600092CFE501EE24FF240AD221E030E00E2CDD
:1010700002C0220F331F0A94E2F728233923232BBF
:1010800009F47BC00091440110E00F7010708E2DA8
:1010900021D290E00817190709F06FC06E2DC40126
:1010A0000DD28350823008F068C08091440190E0F6
:1010B000807F9070803B910509F44DC0813B910584
:1010C00044F48039910569F0803A910509F055C0E2
:1010D0001FC0803D910539F1803E910509F04DC05A
:1010E0002FC06E2DC6019ED181519F4761F06E2D9C
:1010F000C60198D182519F4731F06E2DC60192D121
:1011000083519F47D1F5809130018823E1F715C0C5
:101110006E2DC60187D180529F4779F580913001AD
:101120008823E1F727C06E2DC6017CD180559F47EB
:1011300021F5809130018823E1F7809145011CC0A1
:101140006E2DC6016FD180569F47B9F48091300152
:101150008823E1F70FC06E2DC60164D1892F99272E
:101160002091450130E08217930739F480913001D6
:101170008823E1F78091460188830894E11CF11CE3
:101180002196FBE0EF16F10409F06ECF10922201D8
:10119000FACE20EA3FE0E22FF32F3197F1F7A8953E
:1011A0008A95C9F70895899A889889B910BC88EDFD
:1011B0008AB986E880BD08951F920F920FB60F92EC
:1011C00011248F939F93EF93FF939CB1C59A8EE167
:1011D0008093280180912D01E82FF0E0E95CFD4F1C
:1011E00090838F5F80932D0180912D018F73809369
:1011F0002D0190912D0180912C01981751F480912F
:101200002C018F5F80932C0180912C018F73809330
:101210002C01FF91EF919F918F910F900FBE0F9036
:101220001F9018951F920F920FB60F9211248F9353
:101230009F93EF93FF9390912F0180912E01981728
:10124000B1F0C49A8EE1809327015D9BFECF90910F
:101250002F01E92FF0E0E950FE4F80818CB99F5FAC
:1012600090932F0180912F018F7380932F01FF9115
:10127000EF919F918F910F900FBE0F901F90189537
:1012800090912C0180912D0120E030E0981711F011
:1012900021E030E0C9010895C59A90912C01809118
:1012A0002D019817D1F3C598F89490912C01E92F4E
:1012B000F0E0E95CFD4F80819F5F90932C0190915D
:1012C0002C019F7390932C01789490E00895482FFF
:1012D00080912E0120912F0190E001968F739070E4
:1012E00030E082179307A1F390912F0180912E0196
:1012F000981741F4C49A8EE1809327015D9BFECF3D
:101300004CB90895F89480912E01E82FF0E0E9504F
:10131000FE4F40838F5F80932E0180912E018F734B
:1013200080932E0178940895FC0120E090E003C0A2
:101330008191980F2F5F2617D9F7892F90E08F772B
:1013400090700895CF93DF93F89480EFC0DFC0E0F2
:10135000D0E006C0F0E0E954FE4F80818F77B7DF20
:10136000EC2F609129012196E617A0F387EB91E01D
:10137000DBDFADDF87EFABDF7894DF91CF910895AE
:101380000F931F93142F022F6F70807F862B9FDF88
:10139000812F8F779CDF802F8F7799DF1F910F919F
:1013A00008951F93142F6F70807F862B90DF812FFD
:1013B0008F778DDF1F91089586B320B340B360B35C
:1013C00030E02072307055E0359527955A95E1F759
:1013D00090E08170907033E0880F991F3A95E1F7A3
:1013E000282B50E04078507095E0559547959A9598
:1013F000E1F7242B70E06074707085E07595679557
:101400008A95E1F7262B822F90E0089581B38861B9
:1014100081BB949A9398A09AA89884E690E0B9DE4C
:10142000A89A08956B3018F0E0E0F0E007C0A62F0E
:10143000B0E0AA0FBB1FA80FB91FF8D3CF010895C2
:101440006B3028F4DC01A60FB11D042EF4D30895EF
:10145000662321F4682F85E290E009C0613021F411
:10146000682F8BE390E003C0682F81E590E0DADF1E
:1014700024E08030920710F08FEF93E00895A3E20C
:10148000B0E0D4D3CF010895A3E2B0E00C01DFD3E4
:101490000895682F8B3018F021E030E007C087E610
:1014A00090E0C0DF282F30E021703070C90108952E
:1014B000A1E0B0E0B3D3802D90E008956B3018F038
:1014C00080E090E00895DC01A60FB11DA7D3802D28
:1014D00090E00895282F30E08B3010F0C901089576
:1014E000D901A857BF4F9AD3802D803110F490E0D6
:1014F0000895C90108956B3040F4A62FB0E0AA0FFB
:10150000BB1FA80FB91F0A01A2D308958B30A8F4FE
:10151000E82FF0E0EE0FFF1FCF018B5D9F4FDC0146
:101520000B0195D3CF01855C9F4FDC010A018FD35E
:10153000DF01AF5ABF4F09018AD3089587E880932E
:101540007A0080917A00806480937A0080917A009A
:1015500086FDFCCF82E085BD85E086BD80916E0072
:10156000816080936E00089592E09093B000909314
:10157000B1008CE98093B300E0E7F0E08081826005
:101580008083909380008AE18093810080E49CE9CD
:10159000909387008093860008958630D0F4E82FDA
:1015A000662359F027B181E090E002C0880F991FAF
:1015B000EA95E2F7282B27B9089527B181E090E05A
:1015C00002C0880F991FEA95E2F78095822387B9B8
:1015D0000895893018F5E82FF0E0662379F04AB1D4
:1015E0002AE030E02E1B3F0B81E090E002C0880F24
:1015F000991F2A95E2F7482B4AB908954AB12AE083
:1016000030E02E1B3F0B81E090E002C0880F991F55
:101610002A95E2F7809584238AB908958B30E0F407
:10162000E82FF0E0662361F024B1389781E090E084
:1016300002C0880F991FEA95E2F7282B24B9089574
:1016400024B1389781E090E002C0880F991FEA9595
:10165000E2F78095822384B908958630D0F4E82F8C
:10166000662359F028B181E090E002C0880F991FED
:10167000EA95E2F7282B28B9089528B181E090E097
:1016800002C0880F991FEA95E2F78095822388B9F6
:101690000895893018F5E82FF0E0662379F04BB112
:1016A0002AE030E02E1B3F0B81E090E002C0880F63
:1016B000991F2A95E2F7482B4BB908954BB12AE0C0
:1016C00030E02E1B3F0B81E090E002C0880F991F95
:1016D0002A95E2F7809584238BB908958B30E0F446
:1016E000E82FF0E0662361F025B1389781E090E0C3
:1016F00002C0880F991FEA95E2F7282B25B90895B3
:1017000025B1389781E090E002C0880F991FEA95D3
:10171000E2F78095822385B908951F93182F60E022
:101720000E94CD0A60E0812F0E942D0B1F91089529
:10173000582F863058F426B181E090E002C0880F1F
:10174000991F5A95E2F72823822F10C0893080F420
:1017500049B12AE030E0281B310981E090E002C065
:10176000880F991F2A95E2F74823842F90E0089567
:101770008B3018F080E090E0089543B1282F30E0DE
:101780002850304081E090E002C0880F991F2A95D0
:10179000E2F74823842F90E00895582F863058F4BC
:1017A00028B181E090E002C0880F991F5A95E2F7B6
:1017B0002823822F10C0893080F44BB12AE030E01A
:1017C000281B310981E090E002C0880F991F2A95FB
:1017D000E2F74823842F90E008958B3018F080E0E2
:1017E00090E0089545B1282F30E02850304081E046
:1017F00090E002C0880F991F2A95E2F74823842FB2
:1018000090E008951F93182F682F82E090E00E94C7
:101810005E0A833018F4813030F403C08530A8F5B7
:101820001FC060E02BC0193049F4809180008F7D8B
:1018300080938000809180008F7E0AC01A3051F41E
:10184000809180008F7780938000809180008F7BD3
:101850008093800060E0812F0E94CD0A61E012C079
:10186000193021F480918000806205C01A3029F47B
:101870008091800080688093800061E0812F0E94C9
:10188000CD0A60E0812F0E942D0B1F910895CF9308
:10189000DF9380E384B917B81AB888B18FEF88B99D
:1018A00081E085B980EE8BB9C0E0D0E00E943F0AAC
:1018B00021E030E00C2E02C0220F331F0A94E2F721
:1018C00028233923232B19F08C2F0E94020C2196F8
:1018D000CB30D10559F7DF91CF9108951F920F9228
:1018E0000FB60F921124EF92FF920F931F932F9335
:1018F0003F934F935F936F937F938F939F93AF9398
:10190000BF93CF93DF93EF93FF93809130018823B0
:1019100009F08CC00E943F0A90937802809377026E
:10192000C0E0D0E002E010E06C2FC8010E945E0A27
:101930008330A1F0209177023091780281E090E02D
:101940000C2E02C0880F991F0A94E2F7809590959B
:101950008223932390937802809377022196C93053
:10196000D10511F7C0E0D0E02091770230917802E4
:1019700081E090E00C2E02C0880F991F0A94E2F7D4
:1019800082239323892B51F0FE01EF5FFE4F80816C
:10199000882321F061E08C2F0E942D0B2196C93005
:1019A000D10511F780910A01C82FD0E069E082E0EB
:1019B00090E00E945E0A843049F4CE0134E0880F42
:1019C000991F3A95E1F78053984F0AC088E391E058
:1019D0009C01C29FC001C39F900DD29F900D112406
:1019E000909389008093880080910B01C82FD0E0EC
:1019F0006AE082E090E00E945E0A843049F4CE0101
:101A000024E0880F991F2A95E1F78053984F0AC068
:101A100088E391E09C01C29FC001C39F900DD29FBB
:101A2000900D112490938B0080938A00C0E0D0E049
:101A3000209177023091780281E090E00C2E02C074
:101A4000880F991F0A94E2F782239323892B61F070
:101A500080913001FE01EF5FFE4F9081891721F4E4
:101A600060E08C2F0E942D0B2196C930D10501F723
:101A7000809130018F5F80933001809130018F37EA
:101A800011F410923001809131018C3021F08F5F80
:101A9000809331018AC010923101809128018823FE
:101AA00031F08091280181508093280101C02D9848
:101AB00080912701882331F0809127018150809304
:101AC000270101C02C98809136018A3031F0809135
:101AD00036018F5F8093360168C081E080933601C4
:101AE00000E010E082E0E82E80E0F82E602FC701D1
:101AF0000E945E0A823009F052C00E943F0AC1E093
:101B0000D0E0002E02C0CC0FDD1F0A94E2F78C2338
:101B10009D23892B09F443C0802F0E94980B8823B2
:101B2000C1F080913201909133018C2B9D2B9093C9
:101B300033018093320180913401909135018C23DF
:101B40009D23892B21F560E0802F0E94280A40E028
:101B50001AC080913201909133019E0120953095F9
:101B600028233923309333012093320180913401AB
:101B7000909135018C239D23892B49F062E0802FC1
:101B80000E94280A41E0BC01802F0E9453008091EE
:101B900032019091330190933501809334010F5FAE
:101BA0001F4F0B30110509F0A1CFFF91EF91DF918D
:101BB000CF91BF91AF919F918F917F916F915F91E5
:101BC0004F913F912F911F910F91FF90EF900F90A8
:101BD0000FBE0F901F901895A1E21A2EAA1BBB1BD7
:101BE000FD010DC0AA1FBB1FEE1FFF1FA217B307E9
:101BF000E407F50720F0A21BB30BE40BF50B661FFF
:101C0000771F881F991F1A9469F7609570958095C2
:101C100090959B01AC01BD01CF010895E199FECFE4
:101C2000BFBBAEBBE09A11960DB20895F7DFE02D71
:101C3000F5DFF02D0895E199FECFBFBBAEBB0DBA25
:101C400011960FB6F894E29AE19A0FBE0895F3DF69
:0A1C5000012CF1DF11240895FFCFED
:0C1C5A00FF0000000000000000004040FF
:00000001FF
